:02000000C32912
:08000800F100030E8301F0007A
:100010000408F200BD308107A80F0F28A90AB30A0F
:100020000508AA00731865282406F31C5B28083904
:10003000031949282A05031D50283308153CA10C33
:10004000A00CB301A50B2A282009A2002109A300B6
:100050007314F3152A08A4008C1E3C281819442890
:10006000981844287B08A03E84001A08FA1A3C28F5
:100070008000FB0AFB12FA0A72088400700E8300EB
:10008000F10E710E0B1109001812000018161A0853
:100090003C283308283C03182A287314B3012A2863
:1000A0003308033C0318582833080D3C03182A284A
:1000B0007314B3012A28FF3A2A040839031D68285B
:1000C0001030A500F314B3012A28AA197328B3012C
:1000D000F41F2A28F413831655309D00AA309D0082
:1000E0009C1483122A283308263C03182A28F3106C
:1000F0007310B3012A280F39303EAD003A302D027B
:100100002D08031C0800073E0800AD007D1A0800FA
:100110007E08C03E84002D088000FE0A7E12FD0A83
:100120000800750883169B001C1400001A0883122F
:10013000F6000800831675089B0076089A001C15C7
:10014000F4176400F41BA1289C18A4281C11831226
:1001500008005030852043308520443085203E08FB
:10016000603885203D08603885200D308520F414E6
:1001700029080A3EB700080032080B3C031C08009F
:100180000310320DAC00AC0DAC0D50308520433067
:1001900085204430852000308A002C08D23E031888
:1001A0008A0A82006030852061308520B5280000F1
:1001B000000000006030852062308520B5280000F6
:1001C000000000006030852064308520B5280000E4
:1001D000000000006030852068308520B5280000D0
:1001E000000000006030852070308520B5280000B8
:1001F000000000006130852060308520B5280000B7
:10020000000000006230852060308520B5280000A5
:10021000000000006430852060308520B528000093
:10022000000000006830852060308520B52800007F
:10023000000000007030852060308520B528000067
:10024000000000006030852060308520B5282F0830
:10025000031D2E292130C700C8000800AF0B342928
:100260000830C700C8000800AF0B3B293830C70072
:100270000830C8000800AF0B42290430C7003830EE
:10028000C8000800AF0B49298830C7002130C800DA
:100290000800C601C801C501C70105110000851489
:1002A0000800051D63290130C50803196129C90B20
:1002B000752905114608C51F6029C61F6029450814
:1002C0007F39C90075290130C60803197429C90B83
:1002D000752905154508C51F7329C61F72294608CB
:1002E000C6137329C6177F39C900851C87290130B9
:1002F000C70803198529CA0B992985104808C71F03
:100300008429C81F842947087F39CA0099290130E8
:10031000C80803199829CA0B992985144708C71FCB
:100320009729C81F96294808C8139729C8177F39E5
:10033000CA000800BC0106169D299E299F29A029F4
:10034000A129051A3C14061200008616A729A8291F
:10035000A929AA29AB29051ABC1486120000061780
:10036000B129B229B329B429B529051A3C150613B8
:1003700000008617BB29BC29BD29BE29BF29051A43
:10038000BC158613080083018F3083168100831209
:100390005F30A000213084008001840AA00BCC29AA
:1003A00007309F008316F83085000E308600A53098
:1003B0009800193099008312B03098000B11A030CA
:1003C0008B00A901023085006400A91DE4299A214F
:1003D0003C08093A03191D2C6400291FEC298501EA
:1003E000B60164007A080319102A7C08A03E840034
:1003F0000008AC00FC0AFC12FA030A302C060319B0
:10040000102A0D302C0603190F2AF71A102A780823
:100410004B3E84002C088000F80AF70A102A741456
:10042000F41C1A2A37082902AC00AC1B1A2A7414CF
:100430007415F4107D080319272A0C1E272A7F083B
:10044000C03E840000089900FF0A7F12FD03741C5F
:100450004B2A7419442A77080319462AF9017908A6
:100460004B3E8400F41500084F3A031DF411840A32
:10047000F70B3B2A442A00084B3A031DF411F41DE4
:10048000442AC41F0511462AC41F0515F801F701A7
:100490007410F4107411F31DFD2AF3112908073E9E
:1004A000B800F31B592A2208A6002308A700F31757
:1004B000F12922082606031DF12923082706031D1A
:1004C0006B2A73162908053EB80044080319712ADF
:1004D000C41FFD2AFD2AF3162208A6002308A70040
:1004E000F12985140530AF001030C3000430B0008E
:1004F0002F03B1000310B10DB10D310D3107003ED6
:10050000F50091202206031DA82AF50A9120230652
:10051000031DA92AF50A91207608031D932A430892
:10052000BD04C104AD2AF60B992A4308BD04BF04DB
:10053000AD2AF60B9E2A4308BD04AD2AF60BA32A6A
:100540004309BD05AD2AF60BAD2A4308BD06AD2A09
:10055000F50AF50AF50AB00B812A0310C30CAF0B9C
:10056000762A0530AF001030C3000430B0002F03EE
:10057000053EB1000310B10DB10D310D3107003E44
:10058000F50091202206031DE82AF50A9120230692
:10059000031DE92AF50A91207608031DD32A430892
:1005A000BE04C204ED2AF60BD92A4308BE04C004D7
:1005B000ED2AF60BDE2A4308BE04ED2AF60BE32AE9
:1005C0004309BE05ED2AF60BED2A4308BE06ED2AC7
:1005D000F50AF50AF50AB00BC12A0310C30CAF0BDC
:1005E000B52A0130C4002908103EB9003F08400474
:1005F000031D7416C116A920F129741E102B390889
:100600002902AC00AC1B102B74123F09BD05400938
:10061000BE05BF01C001410842040319C401A9205D
:10062000F31F262B38082902AC00AC1B262B7312B3
:10063000F313C41F8510440B262B4109BD05420945
:10064000BE05C101C201741EC401A92029083B06D0
:100650000319F1293B06BB0051219A214408031DCF
:10066000422B01303C06031DF1298030C400C60135
:10067000C801C501C7018514000005157313B20137
:10068000BC20F129C41FF12903308A00440807392E
:100690008207512B562BFD2B012C102C172C1C2CB8
:1006A0001C2C3C08031DF129C40AF12901303C0629
:1006B000031D682BC40AC601C801C501C701851006
:1006C000000005110A30B200BC20BD01BE01F129B5
:1006D00002303C06031D7E2BC601C801C501C701BF
:1006E0008514000005157313F412B20A0A303202A1
:1006F0000318B201BC208030C400EC2B731FEC2B1C
:10070000B41BB52B04303C06031D912BB50A3508EC
:10071000053C031CB5013508AF0027218030C4001B
:10072000912B08303C06031DB52B3408F50005302D
:1007300035060319A72B2208F6009A20F50A23088C
:10074000F6009A20F50A3508F6009A20A92BF60142
:100750009A208030C400C601C801C501C7018514B4
:10076000000005157313F412EC2BF41AEC2BF4169D
:10077000B4170430B0003208B1000310B10DB10D50
:10078000310D3107003EF50091200038031DCB2BC1
:100790007508B400D42B2206031DD42BF50A912032
:1007A00023060319E42BD52BF50AF50AF50AB00B3D
:1007B000C42B8514B41BDF2B0530B500EC2B38306F
:1007C000C6000430C500EC2B7503B400F50A912077
:1007D000B500AF002721EC2BF31CF1298330C400B6
:1007E000C601C801C501C70105110000851029080F
:1007F0000A3EBA007313F412F1293C080319C4012C
:10080000F1293A082902AC00AC1F0B2C731EF12908
:100810008430C400F129051573138030C400F12918
:10082000731AF129731785148030C400F1293C082C
:10083000031DF129C40AF129F12951211C30C600F8
:100840001C30C5001C30C8001C30C70064002908DB
:100850003B060319262C3B06BB0051219A213C087C
:10086000023A031D262C2830B0000030F500F601B6
:100870009A200330F507B00B372CC601C801C5011B
:04088000C701E129A2
:02400E00663F0B
:10420000030021000100430019000000000000002D
:104210000000000000000000030022000100430035
:104220001800000000000000000000000000000076
:10423000030023000100430006000000000000000E
:104240000000000000000000030024000100430003
:104250000700000000000000000000000000000057
:1042600003002500010043002100040043000C006E
:104270000200430003000300030026000100430086
:104280002200040043000C0002004300030003006E
:1042900003002700010043002300040043000C003A
:1042A0000200430003000300030028000100430054
:1042B0002400040043000C0002004300030003003C
:1042C00003002900010043002500040043000C0006
:1042D000020043000300030003002A000100430022
:1042E0002600040043000C0002004300030003000A
:00000001FF
